:1000000065C0BFC17DC07CC07BC07AC079C078C0EC
:1000100077C076C075C074C073C072C071C070C044
:100020006FC06EC06DC0090222000101008032095C
:100030000400000103000000092101010001220069
:10004000000705810308000A04030904180372006D
:100050006100700068006E00650074002E006E0084
:10006000650074001603470043002F004E00360061
:1000700034005F005500530042000A033600300090
:1000800031003100120101010000000881179A0AB5
:1000900001010102030105010905A1010901A100F6
:1000A00005010930093109330934093509361500CC
:1000B00026FF00750895068102C00509190129105F
:1000C00015002501750195108102C00011241FBE85
:1000D000CFE5D4E0DEBFCDBF10E0A0E6B0E0ECE2BB
:1000E000F0E102C005900D92A239B107D9F710E0F6
:1000F000A2E9B0E001C01D92AE3FB107E1F740C3F5
:100100007FCF82E990E08093F2000B968093E60027
:1001100085B7836085BF8BB780648BBF08951F93BD
:10012000DC01162F693008F018E09091AA0090FFCA
:1001300002C023EC01C02BE48091620087FF04C061
:100140009F5F9093AA0003C08FEF8093620020937B
:10015000E700912FE8EEF0E002C08D91819391507D
:10016000E0F7612F88EE90E0BED21C5F1093620032
:100170001F9108950F931F938091F700882309F42E
:1001800096C0982F935097FD90C0E2E9F0E08091DF
:10019000E600E82FEF5F8091F4008D3209F07FC018
:1001A000983009F07CC08081807609F074C010928C
:1001B000E1008181882321F41092E20022E05CC0FA
:1001C000853021F482818093F80055C08630F1F5A6
:1001D0008381813039F42091F9008091E40090917D
:1001E000E50032C0823021F486E290E022E22CC0A9
:1001F0008330C9F48281882321F488E490E024E0EC
:1002000023C0813021F48CE490E028E11DC08230CD
:1002100021F484E690E026E117C0833061F48AE798
:1002200090E02AE011C0813221F488E390E029E0D7
:100230000BC0823219F020E030EC1FC02091E300A7
:100240008091FC009091FD0030EC19C0883029F4B9
:1002500021E030E88BEF90E012C0893021F48281F8
:100260008093FB0008C08A3011F421E005C08B3078
:1002700011F41092AA0020E030E881EE90E0909313
:10028000F6008093F5008781882359F486818217D0
:1002900040F4282F06C0CF013FD2282F01C020E014
:1002A00030E83093A800209360001092F7009091FE
:1002B00060009F3F09F44BC08091610087FF47C0F9
:1002C000692F993008F068E0961B90936000809148
:1002D000A80080FF02C003EC01C00BE48F5F809395
:1002E000A800E091F500F091F60086FD04C0962F7D
:1002F000A9EDB0E017C04091E300262FA9EDB0E0D2
:100300000CC03491CD01019650E0EF33F50711F4A4
:100310004C9301C03C93DC013196215090F704C00E
:1003200081918D939150E0F7F093F600E093F50002
:100330007727162F89ED90E0D6D1183018F48FEF7B
:10034000809360000093D8001C5F1093610080B31D
:10035000857019F01092A90011C08091A90088231E
:1003600069F494E680B3857049F49150D9F781E03F
:100370008093A9001092F8001092F3001F910F9142
:1003800008950F930FB70F93809BFECF809B06C0FD
:10039000809B04C0809B02C0000000C01F933F935D
:1003A0002F9331E014E000B3102710FD32E0102F3E
:1003B0003A95C9F700FDE7C000B3102717952FE75E
:1003C0002795DF9310B3012707952795CF93C09109
:1003D000F20000B31027179527953BE0D0E04F932C
:1003E00010B30127079527954FEF000055C0809B5C
:1003F000FECF809B06C0809B04C0809B02C0000093
:1004000000C0DF9100C0CDCF10B3157079F1407CF2
:100410002C6F13C000B3057049F141782C6F15C0E3
:10042000057021F1102F2C6F00B319C000B30570B7
:10043000E9F04E7F2C6F18C038F300B30570B1F0AF
:10044000102717952795243028F310B30127079517
:100450002795422749934FEF00B3243008F3102724
:1004600017952795243010F310B31570E1F101278B
:10047000079527952430F0F000B30570A1F11027FF
:10048000179527952430E0F010B30127079527959D
:100490003A9541F12430D0F000B3057021F11027D6
:1004A000179527952430C0F010B30127079527959D
:1004B0002430C2CF10B31570B1F04C7F2C6FDCCF5D
:1004C00000B3057081F0487F2C6FDECF10B315703C
:1004D00051F0407F2C6FE0CF00B3057021F0407EDB
:1004E0002C6FE2CF3DC03C2FC091F2003C1B00E4DA
:1004F00033300ABFA8F108811981412F1F7720915D
:10050000F3000D3289F1013E79F10936C1F0077728
:10051000033431F51091FA00112311F10091F70025
:100520000030D1F53430DAF13093F7001093F40055
:100530000091E600C093E6000093F20030C012176D
:1005400079F447FD3AC0309161003F3F29F10FEF48
:1005500000936100C8EDD0E025C000270093FA00A9
:100560004F91CF91DF910FC01217B9F70093FA00A6
:100570000FEF00936000009361004F91CF910AB795
:1005800006FD35CFDF9100E40ABF2F913F911F9107
:100590000F910FBF0F911895C4E6D0E002C0C3E6DB
:1005A000D0E032E05F9302B30A7F016002BB55E006
:1005B00011B3156011BB20E819C0309162003F3FB4
:1005C00059F30FEF00936200C7EED0E0EBCF0527A1
:1005D00010E002BB10C0052710E0089402BB13C056
:1005E000052710E015C0052710E019C020FF0527DA
:1005F00002BB279517951C3F50F720FF052727952D
:1006000002BB17951C3F38F720FF05272795179544
:1006100002BB1C3F28F720FF0527279517951C3F95
:1006200002BB08F700C0499120FF052702BB2795B0
:1006300017951C3F80F520FF0527279502BB1795CE
:100640001C3F68F520FF05272795179502BB1C3F27
:1006500058F520FF0527279517951C3F02BB38F555
:10066000242F3A9519F60A7F5F9102BB32E03A9542
:10067000F1F71091F800C656D04011F01093F30036
:10068000016011B31A7F02BB0A7F4F91CF9111BB5A
:1006900002BBDF9178CF052710E002BBCACF052748
:1006A00010E0089402BBCDCF052710E0CFCF05277F
:1006B00010E0D3CFA82FB92F8FEF9FEF41E050EA82
:1006C000615070F02D9138E0722F782796958795BC
:1006D000269570FF02C0842795273A95A9F7F0CF99
:1006E000809590950895E6DF8D939D93089514BAB3
:1006F0008FEF85BB88EF82BB85E081BB9EEF8FEFDC
:100700009150F1F78150E1F711BA85E083BF8FE096
:1007100085BD84EC83BD0895FC012DEA30E0309363
:10072000F6002093F50080818076803231F581815A
:10073000813081F4E091AB00F091AC000088F18948
:10074000E02DC9010995E091AB00F091AC008081EA
:1007500099270895823049F485EB90E09093F60054
:100760008093F50081E090E008958A3031F4838130
:100770008093B50080E090E0089580E090E00895D7
:10078000CFE5D4E0DEBFCDBFB2DFB9D2FC0190939C
:10079000AC008093AB000284F385E02D0995E091D5
:1007A000AB00F091AC000288F389E02D0995882315
:1007B000A1F41ED4FC019093AC008093AB000284A2
:1007C000F385E02D0995E091AB00F091AC00028833
:1007D000F389E02D09958823C1F286E990E0909392
:1007E000FD008093FC0012D48093E30084E890E045
:1007F0009093E5008093E40090D28093F90077DF36
:10080000E091AB00F091AC000284F385E02D0995F6
:1008100088E190E02FE00FB6F894A89581BD0FBE57
:1008200021BD6FDC789400E011E0FF2401C010E0EE
:10083000A895A0DC112341F0E091AB00F091AC0051
:100840000484F585E02D099508B600FE0EC081E010
:1008500088BF8091B500882341F094E09F1518F07F
:10086000F82E01E002C08BEFF80E08B607FE17C0A5
:1008700080E888BF0023A9F4E091AB00F091AC00C0
:100880000484F585E02D0995E091AB00F091AC0072
:100890000684F785E02D09958823D9F4C8CF002375
:1008A00031F2809162008F3F11F6E091AB00F09140
:1008B000AC000088F189E02D8DEA90E00995E09187
:1008C000AB00F091AC0060818DEA90E028DC00E0A4
:1008D000AECF01E0E6CF009741F0FC01A6EBB0E01F
:1008E00088E00D9001928150E1F7AEEBB0E0E6EBCD
:1008F000F0E088E001900D928150E1F70895809139
:10090000790090917A00892B39F010927A00109238
:10091000790021E030E00BC048E050E06EEB70E081
:1009200086EB90E076D3282F332727FD3095C90139
:1009300008950F931F93CF93DF93CDB7DEB7C954BC
:10094000D0400FB6F894DEBF0FBECDBF80E0FE01F1
:100950003996EF93FF9300E810E41023A9F000000C
:10096000A59A000000000000000000000000000048
:10097000000000000000A59838E03A95F1F700006B
:100980000000069561F0E8CFA59A3BE03A95F1F7B3
:100990000000A59800000000069509F0DDCFA5989D
:1009A00000E813E01023A9F00000A59A0000000061
:1009B0000000000000000000000000000000000037
:1009C000A59838E03A95F1F700000000069561F02F
:1009D000E8CFA59A3BE03A95F1F70000A598000012
:1009E0000000069509F0DDCFA59800E8182F102328
:1009F000A9F00000A59A000000000000000000001F
:100A000000000000000000000000A59838E03A95C2
:100A1000F1F700000000069561F0E8CFA59A3BE0F1
:100A20003A95F1F70000A59800000000069509F03E
:100A3000DDCFA5980000000000000000A59A00008E
:100A4000000000000000A59830E40FE30A9529F1AA
:100A500013B31072D9F7C198000000000000000025
:100A60000000000000000000000000000000000086
:100A700000000000000023B3C19A207221933A9530
:100A800039F00FE30A9549F023B32072F1F6FACF5B
:100A9000882705C0C19A832F02C088278095FF91BF
:100AA000EF91C1988F3F21F481E08093C600F9C097
:100AB00088E0FE01319611928A95E9F7498120E09C
:100AC00030E060E870E0FE0179968191882339F08A
:100AD000CB01022E02C0959587950A94E2F7482B28
:100AE0002F5F3F4F2830310581F749834A8120E04D
:100AF00030E060E870E0FE01B1968191882339F022
:100B0000CB01022E02C0959587950A94E2F7482BF7
:100B10002F5F3F4F2830310581F740954A834B8145
:100B200020E030E060E870E0FE01B9968191882312
:100B300039F0CB01022E02C0959587950A94E2F711
:100B4000482B2F5F3F4F2830310581F74B834C8175
:100B500020E030E060E870E0FE01F19681918823AA
:100B600011F080E007C0CB01022E02C09595879559
:100B70000A94E2F7482B2F5F3F4F2830310571F779
:100B80004C834D8120E030E060E870E0FE01F99692
:100B90008191882339F0CB01022E02C0959587956B
:100BA0000A94E2F7482B2F5F3F4F2830310581F739
:100BB00040954D834E8120E030E060E870E0FE011A
:100BC000EF5BFF4F8191882339F0CB01022E02C0E9
:100BD000959587950A94E2F7482B2F5F3F4F283071
:100BE000310581F740954E834F8120E030E061E090
:100BF00070E0FE013C968191882339F0CB01022EF2
:100C000002C0880F991F0A94E2F7482B2F5F3F4FCD
:100C10002530310581F720E030E060E270E0FE0130
:100C200072968191882339F0CB01022E02C0880F81
:100C3000991F0A94E2F7482B2F5F3F4F233031056D
:100C400081F74F83488520E030E061E070E0FE01ED
:100C500075968191882339F0CB01022E02C0880F4E
:100C6000991F0A94E2F7482B2F5F3F4F243031053C
:100C700081F7488789818093B6008A818093B70085
:100C80008B818093B8008C818093B9008D81809393
:100C9000BA008E818093BB008F818093BC0040930B
:100CA000BD00C75BDF4F0FB6F894DEBF0FBECDBFF0
:100CB000DF91CF911F910F9108951F9310E080E075
:100CC00090E00197F1F71092C60033DE8091C600E4
:100CD000882319F481E090E005C01F5F1F3079F789
:100CE00080E090E01F9108951F931FB7F894B99A80
:100CF000C198A598AD981DDE1FBF1F91089586E984
:100D000090E090936A008093690080D1909368008E
:100D10008093670085E690E0089582E190E0089571
:100D20000F931F93CF93DF93CDB7DEB7C154D0405D
:100D30000FB6F894DEBF0FBECDBF91E0FE01319635
:100D4000EF93FF9300E8192F1023A9F00000A59A54
:100D50000000000000000000000000000000000093
:100D600000000000A59838E03A95F1F70000000077
:100D7000069561F0E8CFA59A3BE03A95F1F70000BF
:100D8000A59800000000069509F0DDCFA5980000A9
:100D90000000000000000000000000000000000053
:100DA000A59A0000000000000000A59830E20FEFB7
:100DB0000A9529F113B31072D9F7C1980000000009
:100DC0000000000000000000000000000000000023
:100DD0000000000000000000000023B3C19A207250
:100DE00021933A9539F00FEF0A9549F023B3207219
:100DF000F1F6FACF882705C0C19A832F02C0882751
:100E00008095FF91EF91C1988F3F19F49093D7008F
:100E100093C020E030E070E041E050E08191882311
:100E200039F0CA01022E02C0880F991F0A94E2F716
:100E3000782B2F5F3F4F2430310581F720E030E0E1
:100E400040E150E0FE013D968191882339F0CA01CE
:100E5000022E02C0880F991F0A94E2F7782B2F5FA9
:100E60003F4F2430310581F79B85911191E08C85AE
:100E7000811182E0592F582B20E030E060E0A0E89B
:100E8000B0E0FE0171968191882339F0CD01022EE8
:100E900002C0959587950A94E2F7682B2F5F3F4F24
:100EA0002830310581F720E030E040E0A0E8B0E0F4
:100EB000FE0179968191882339F0CD01022E02C07E
:100EC000959587950A94E2F7482B2F5F3F4F28307E
:100ED000310581F761586093C7008FE7982F941B05
:100EE0009093C8008093C9008093CA008093CB0080
:100EF0008093CC007093CD005093CE008D818823D9
:100F000019F054605093CE008E81882329F080918F
:100F1000CE0088608093CE008F81882329F0809155
:100F2000CE0080618093CE008885882329F080914F
:100F3000CE0080628093CE00CF5BDF4F0FB6F89477
:100F4000DEBF0FBECDBFDF91CF911F910F910895EE
:100F50001F931FB7F894B99AC198A598AD98E0DE91
:100F60001FBF1F9108951F9310E080E090E001974C
:100F7000F1F71092D700D4DE8091D700882319F4BE
:100F800081E090E005C01F5F1F3079F780E090E0BE
:100F90001F910895009741F0FC01A7ECB0E088E0B4
:100FA0000D9001928150E1F7AFECB0E0E7ECF0E09A
:100FB00088E001900D928150E1F7089580918F00B3
:100FC00090919000892B39F01092900010928F0030
:100FD00021E030E00BC048E050E06FEC70E087ECBF
:100FE00090E017D0282F332727FD3095C9010895A9
:100FF00086E990E09093800080937F0007D09093E3
:101000007E0080937D008BE790E0089585E390E07B
:101010000895FB01DC0104C08D910190801921F439
:0C10200041505040C8F7881B990B089500
:10102C00FFFFFFD25A08000000000000000000740F
:10103C000699047F046B045D0601000800000000A3
:10104C000000000000A8079006DE07CA07B30701DE
:02105C00000092
:00000001FF
